:100000000C9438000C9453000C9453000C9453003F
:100010000C9453000C9453000C9410160C94530041
:100020000C9453000C9453000C94E3150C9453005F
:100030000C94DC140C9453000C9453000C94530057
:100040000C9453000C9499030C9453000C9453009B
:100050000C94DA120C9453000C9453000C9453003B
:100060000C9453000C9453000C9453000C945300C4
:1000700011241FBECFEFD4E0DEBFCDBF12E0A0E061
:10008000B1E0E2E4FEE202C005900D92A438B107AF
:10009000D9F713E0A4E8B2E001C01D92A539B10779
:1000A000E1F70C9476000C940000CF93DF93CDB76A
:1000B000DEB7E1E3F0E080E18083E4E3F0E08FEF9E
:1000C0008083EAE3F0E08EE28083ABE3B0E0EBE331
:1000D000F0E0808182608C93ABE3B0E0EBE3F0E092
:1000E000808180628C93DF91CF910895CF93DF93CD
:1000F000CDB7DEB725970FB6F894DEBF0FBECDBFE4
:100100000E9455000E9476030E940D117894A5E389
:10011000B0E0E5E3F0E0808181608C930E944D03C4
:100120000E9461070E9474060E94C1050E94DF03BD
:100130000E942B0500C0809186028130C9F4109284
:10014000860289818F5F89830E944811198280917C
:100150009302882319F40E948F1506C08091010133
:10016000823014F00E948F150E94BA140E94C914A4
:1001700080919C02813099F5A5E3B0E0E5E3F0E0E1
:10018000808184608C930E94141080919302882354
:1001900069F40E94330B0E94670C0E941E0A0E94A1
:1001A00081090E94FD070E94560612C0809101013C
:1001B000823034F00E941E0A0E9481090E94560675
:1001C00080910101833024F00E94330B0E94670C60
:1001D000A5E3B0E0E5E3F0E080818B7F8C93809134
:1001E0008402813071F510928402809193028823F9
:1001F00019F40E942B0506C080910101833014F090
:100200000E942B058091900290919102019690930B
:1002100091028093900280919002909191028C3390
:10022000910569F480918E0290918F0201969093CE
:100230008F0280938E0210929102109290020E947F
:10024000830680918502813009F075CF1092850276
:1002500080919A02282F332727FD30953D832C83E8
:100260008C819D818130910531F02C813D8122303E
:10027000310539F00BC00E94150582E080939A0287
:1002800005C00E94200581E080939A02809193022C
:10029000813009F050CF80919202813009F04BCF2C
:1002A0001092920280910101282F332727FD30956B
:1002B0003B832A838A819B8181309105C1F02A8109
:1002C0003B81223031052CF48A819B81009761F0BB
:1002D00032CF2A813B812230310571F08A819B81A6
:1002E00083309105B1F027CF0E94150524CF0E94DD
:1002F00020050E94390E1FCF0E94200564E084E093
:100300000E94B5010E9461070E9474060E94C10507
:1003100012CF0E94200564E084E00E94B5010E9493
:1003200061070E9474060E94C1050E942B0503CF3D
:10033000CF93DF93CDB7DEB764E084E00E94B501D0
:100340006CE480E00E94B5011092860280918602E2
:100350008823E1F36AE08CE60E94B50160E085E065
:100360000E94B501DF91CF910895CF93DF93CDB770
:10037000DEB724970FB6F894DEBF0FBECDBF8B83D8
:100380006C83ABE3B0E0EBE3F0E080818D7F8C9396
:1003900087E08A8340C0ABE3B0E0EBE3F0E080812C
:1003A000877F8C9300000000000000008A81282FC6
:1003B000332727FD309581E090E0022E02C0880FA0
:1003C000991F0A94E2F7982F8B8189238983898169
:1003D000882341F0ABE3B0E0EBE3F0E080818460A0
:1003E0008C9307C0ABE3B0E0EBE3F0E080818B7F60
:1003F0008C930000000000000000ABE3B0E0EBE3F2
:10040000F0E0808188608C93000000000000000014
:100410008A8181508A838A8188230CF0BCCF87E04F
:100420008A8340C0ABE3B0E0EBE3F0E08081877FFC
:100430008C9300000000000000008A81282F3327E1
:1004400027FD309581E090E0022E02C0880F991FB1
:100450000A94E2F7982F8C818923898389818823E4
:1004600041F0ABE3B0E0EBE3F0E0808184608C939B
:1004700007C0ABE3B0E0EBE3F0E080818B7F8C93CF
:100480000000000000000000ABE3B0E0EBE3F0E0B0
:10049000808188608C9300000000000000008A8149
:1004A00081508A838A8188230CF0BCCFABE3B0E013
:1004B000EBE3F0E08081877F8C93ABE3B0E0EBE38C
:1004C000F0E080818B7F8C93ABE3B0E0EBE3F0E076
:1004D000808182608C9324960FB6F894DEBF0FBEA5
:1004E000CDBFDF91CF910895CF93DF93CDB7DEB726
:1004F00024970FB6F894DEBF0FBECDBF8C83ABE35D
:10050000B0E0EBE3F0E080818D7F8C9387E08A831D
:100510004CC0ABE3B0E0EBE3F0E08081877F8C93ED
:1005200000000000000000000000000000000000CB
:100530008A81282F332727FD309581E090E0022E15
:1005400002C0880F991F0A94E2F7982F8C818923A3
:100550008B838B81181644F4ABE3B0E0EBE3F0E05F
:10056000808184608C9307C0ABE3B0E0EBE3F0E004
:1005700080818B7F8C930000000000000000000051
:10058000000000000000ABE3B0E0EBE3F0E08081AE
:1005900088608C9300000000000000000000000054
:1005A000000000008A8181508A838A8188230CF0B0
:1005B000B0CF1B82ABE3B0E0EBE3F0E08081877F5C
:1005C0008C9300000000000000000000000000000C
:1005D000000087E08A833DC0ABE3B0E0EBE3F0E0EE
:1005E000808188608C93E9E3F0E080818983898150
:1005F000992780719070181619068CF48A81282F1B
:10060000332727FD309581E090E0022E02C0880F4D
:10061000991F0A94E2F7982F8B81892B8B83000016
:100620000000000000000000000000000000ABE33C
:10063000B0E0EBE3F0E08081877F8C930000000066
:100640000000000000000000000000008A818150CE
:100650008A838A8188230CF0BFCFABE3B0E0EBE361
:10066000F0E08081877F8C93ABE3B0E0EBE3F0E0D8
:1006700080818B7F8C93ABE3B0E0EBE3F0E0808193
:1006800082608C938B81992724960FB6F894DEBFF5
:100690000FBECDBFDF91CF910895CF93DF93CDB73C
:1006A000DEB70E9498011092840280918402882310
:1006B000E1F30E9468050E94390E10928402809135
:1006C00084028823E1F310928402809184028823BB
:1006D000E1F31092840264E084E00E94B5016CE4CE
:1006E00080E00E94B501DF91CF910895CF93DF9311
:1006F000CDB7DEB7E3E5F0E082E08083EEE4F0E042
:1007000082E48083E9E5F0E08AE18083E7E4F0E0D9
:1007100086E08083E2E4F0E080EF8083EAE8F0E0C6
:1007200083E48083EDE7F0E080E28083DF91CF9186
:1007300008951F920F920FB60F9211248F93CF93AB
:10074000DF93CDB7DEB7809188028F5F80938802F8
:1007500080918802883459F581E080938702109255
:100760008802809150038F5F8093500380915003E3
:10077000843641F41092500381E08093840281E03A
:100780008093850280915003823319F481E0809335
:10079000850280914F038F5F80934F0380914F03B9
:1007A0008A3029F410924F0381E080938602DF9112
:1007B000CF918F910F900FBE0F901F901895CF93F0
:1007C000DF93CDB7DEB762E480E00E94B5011092FE
:1007D0008402809184028823E1F31092840266E708
:1007E00089E00E94B50110928602809186028823DA
:1007F000E1F3109286021092510316C080915103CA
:10080000682F8AE00E94B501809151039927FC016D
:10081000E95CFE4F8081682F8BE00E94B5018091DA
:1008200051038F5F8093510380915103863330F3DE
:1008300060EA88E00E94B5011092860280918602EB
:100840008823E1F310928402809184028823E1F3EB
:100850001092840267E789E00E94B5011092860237
:10086000809186028823E1F3109286021092510350
:1008700016C080915103682F8AE00E94B5018091D3
:1008800051039927FC01E958FE4F8081682F8BE0C6
:100890000E94B501809151038F5F80935103809135
:1008A0005103863330F360EA88E00E94B50110926C
:1008B0008602809186028823E1F31092840280915F
:1008C00084028823E1F31092840268E789E00E94A1
:1008D000B50110928602809186028823E1F310927E
:1008E00086021092510316C080915103682F8AE04E
:1008F0000E94B501809151039927FC01E954FE4FF4
:100900008081682F8BE00E94B501809151038F5F39
:100910008093510380915103863330F360EA88E07D
:100920000E94B50110928602809186028823E1F32D
:1009300010928402809184028823E1F31092840251
:1009400069E789E00E94B5011092860280918602D3
:100950008823E1F3109286021092510316C0809111
:100960005103682F8AE00E94B501809151039927B5
:10097000FC01E950FE4F8081682F8BE00E94B50199
:10098000809151038F5F809351038091510386338F
:1009900030F360EA88E00E94B501109286028091EF
:1009A00086028823E1F310928402809184028823D6
:1009B000E1F3109284026AE789E00E94B501109287
:1009C0008602809186028823E1F3109286021092BB
:1009D000510316C080915103682F8AE00E94B5012F
:1009E000809151039927FC01E95CFD4F8081682FBC
:1009F0008BE00E94B501809151038F5F809351037A
:100A000080915103863330F360EA88E00E94B5019B
:100A100010928602809186028823E1F36CE480E0E4
:100A20000E94B501DF91CF910895CF93DF93CDB7A9
:100A3000DEB762E480E00E94B501DF91CF910895B6
:100A4000CF93DF93CDB7DEB76CE480E00E94B501B1
:100A5000DF91CF910895CF93DF93CDB7DEB789EDC6
:100A60008093510313C060E085E00E94B50180913E
:100A70005103682F86E00E94B50164E587E00E947B
:100A8000B501809151038F5F809351038091510391
:100A90008C3D48F385EE8093510313C060E085E000
:100AA0000E94B50180915103682F86E00E94B50134
:100AB00064E587E00E94B501809151038F5F8093C8
:100AC000510380915103883E48F3DF91CF910895FF
:100AD000CF93DF93CDB7DEB764970FB6F894DEBF40
:100AE0000FBECDBF8DE589838EE58A838FE58B832D
:100AF00089E48C838BE58D838DE18E838CE58F83F8
:100B0000188680E2898789E28A8786E38B8781E479
:100B10008C878AE08D8781E48E8785E08F8786E2E7
:100B2000888B20E1CE010196AC0162E087E00E9453
:100B3000EC0564960FB6F894DEBF0FBECDBFDF9113
:100B4000CF910895CF93DF93CDB7DEB760E085E016
:100B50000E94B5016FEC86E00E94B5016CE887E069
:100B60000E94B50161E085E00E94B5016BE086E07E
:100B70000E94B5016DE887E00E94B501DF91CF9139
:100B80000895CF93DF93CDB7DEB760E085E00E9494
:100B9000B50160E286E00E94B50160E887E00E944E
:100BA000B50160E085E00E94B5016EE386E00E9439
:100BB000B50164E887E00E94B50160E085E00E942D
:100BC000B5016CE586E00E94B50168E887E00E9407
:100BD000B501DF91CF910895CF93DF93CDB7DEB705
:100BE0002D970FB6F894DEBF0FBECDBF89876A87F9
:100BF0005C874B872D878A85282F33278EE190E0ED
:100C0000A901489F9001499F300D589F300D112434
:100C100089859927820F931F98878F838D85282F29
:100C200033278F819885820F931F9E838D83109227
:100C300051038F8198859C838B8328C08B818A8305
:100C40008B819C81892F99278983698185E00E9406
:100C5000B5016A8186E00E94B50140915103842F5D
:100C600099279C018B859C85F901E80FF91F8081EC
:100C7000982F842F8F5F80935103692F87E00E9404
:100C8000B5018B819C8101969C838B832B813C8158
:100C90008D819E812817390788F22D960FB6F8941A
:100CA000DEBF0FBECDBFDF91CF910895CF93DF930D
:100CB000CDB7DEB78091680390916903843B9105BD
:100CC00044F480919A02882361F481E080939A022F
:100CD00008C080919A02181614F40E942005109200
:100CE0009A02DF91CF910895CF93DF93CDB7DEB70E
:100CF00086E091E025E0AC016EE087E10E94EC0522
:100D0000DF91CF9108950F931F93CF93DF93CDB7CA
:100D1000DEB729970FB6F894DEBF0FBECDBF188699
:100D20008AE0898720918E0230918F02CE0102964F
:100D30004AE050E0BC01C9010E94C916CE010296EA
:100D4000DC01FD0101900020E9F73197CF018A1BFA
:100D50009B0B8983109251031CC080915103082F73
:100D6000112780915103282F3327CE010296FC01D1
:100D7000E20FF31F80810E948A08282FCE0105967A
:100D8000FC01E00FF11F2083809151038F5F80935E
:100D9000510380915103282F33278981992787FD9B
:100DA000909528173907CCF280918E0290918F028E
:100DB0008A3091058CF4CE01089621E0AC016EE0FA
:100DC00087E10E94EC05CE01059621E0AC016EE0C2
:100DD00088E10E94EC0508C0CE01059622E0AC0136
:100DE0006EE087E10E94EC05209190023091910223
:100DF000CE0102964AE050E0BC01C9010E94C9162A
:100E0000CE010296DC01FD0101900020E9F7319747
:100E1000CF018A1B9B0B8983109251031CC08091C8
:100E20005103082F112780915103282F3327CE011A
:100E30000296FC01E20FF31F80810E948A08282F8E
:100E4000CE010596FC01E00FF11F20838091510334
:100E50008F5F8093510380915103282F332789811D
:100E6000992787FD909528173907CCF28091900239
:100E7000909191028A3091058CF4CE01099621E07F
:100E8000AC016EE08AE10E94EC05CE01059621E0FE
:100E9000AC016EE08BE10E94EC0508C0CE01059626
:100EA00022E0AC016EE08AE10E94EC0529960FB6C3
:100EB000F894DEBF0FBECDBFDF91CF911F910F9190
:100EC0000895CF93DF93CDB7DEB782E091E024E0C1
:100ED000AC016EE082E00E94EC05DF91CF910895B5
:100EE0000F931F93CF93DF93CDB7DEB761970FB604
:100EF000F894DEBF0FBECDBFCE010A969E878D87C8
:100F0000E7E7F2E0F88BEF87F3E0F98BEF85F889FC
:100F100000808F8598890196988B8F87ED85FE8557
:100F200000828D859E8501969E878D879989915037
:100F3000998BE989EE2351F720916A0330916B0375
:100F4000CE0102964AE050E0BC01C9010E94C916D8
:100F5000CE010296DC01FD0101900020E9F73197F6
:100F6000CF018A1B9B0B8983109251031CC0809177
:100F70005103082F112780915103282F3327CE01C9
:100F80000296FC01E20FF31F80810E948A08282F3D
:100F9000CE010696FC01E00FF11F208380915103E2
:100FA0008F5F8093510380915103282F33278981CC
:100FB000992787FD909528173907CCF2CE010A961C
:100FC00023E0AC016DE08DE00E94EC052981998160
:100FD00080E1382F391BCE010696AC016DE0832FDE
:100FE0000E94EC0561960FB6F894DEBF0FBECDBF30
:100FF000DF91CF911F910F9108950F931F93CF937E
:10100000DF93CDB7DEB761970FB6F894DEBF0FBEA2
:10101000CDBFCE010A969E878D87EAE7F2E0F88B76
:10102000EF87F3E0F98BEF85F88900808F85988949
:101030000196988B8F87ED85FE8500828D859E8534
:1010400001969E878D8799899150998BE989EE2326
:1010500051F72091640330916503CE0102964AE076
:1010600050E0BC01C9010E94C916CE010296DC0104
:10107000FD0101900020E9F73197CF018A1B9B0BFE
:101080008983109251031CC080915103082F1127AE
:1010900080915103282F3327CE010296FC01E20FE5
:1010A000F31F80810E948A08282FCE010696FC013A
:1010B000E00FF11F2083809151038F5F80935103D4
:1010C00080915103282F33278981992787FD909597
:1010D00028173907CCF2CE010A9623E0AC016EE066
:1010E0008DE00E94EC052981998180E1382F391B20
:1010F000CE010696AC016EE0832F0E94EC0561964E
:101100000FB6F894DEBF0FBECDBFDF91CF911F9118
:101110000F910895CF93DF93CDB7DEB722970FB627
:10112000F894DEBF0FBECDBF8A838A818D3219F459
:1011300089E4898309C08A81803319F48AE089832C
:1011400003C08A81805389838981992787FD90957F
:1011500022960FB6F894DEBF0FBECDBFDF91CF91C0
:1011600008950F931F93CF93DF93CDB7DEB76097AA
:101170000FB6F894DEBF0FBECDBF85E0FE013C96F2
:10118000DF01982F1D929A95E9F72091B0023091D6
:10119000B102CE0102964AE050E0BC01C9010E94B2
:1011A000C916CE010296DC01FD0101900020E9F78D
:1011B0003197CF018A1B9B0B8983109251031CC06E
:1011C00080915103082F112780915103282F332735
:1011D000CE010296FC01E20FF31F80810E948A0873
:1011E000282FCE010796FC01E00FF11F208380918C
:1011F00051038F5F8093510380915103282F332730
:101200008981992787FD909528173907CCF2CE015F
:101210000C9624E0AC0167E089E10E94EC0529818D
:1012200099818CE1382F391BCE010796AC0167E01C
:10123000832F0E94EC058091B0029091B1021816A4
:101240001906C4F460E085E00E94B5016FEC86E009
:101250000E94B5016CE887E00E94B50161E085E07D
:101260000E94B5016BE086E00E94B50160E087E076
:101270000E94B5018091B0029091B1029923C4F40B
:1012800060E085E00E94B5016FEC86E00E94B50148
:1012900060E087E00E94B50161E085E00E94B50151
:1012A0006BE086E00E94B5016DE887E00E94B50121
:1012B0008091B0029091B1020097C1F460E085E0A6
:1012C0000E94B5016FEC86E00E94B50160E087E006
:1012D0000E94B50161E085E00E94B5016BE086E007
:1012E0000E94B50160E087E00E94B50160960FB6EC
:1012F000F894DEBF0FBECDBFDF91CF911F910F914C
:1013000008950F931F93CF93DF93CDB7DEB7659703
:101310000FB6F894DEBF0FBECDBFCE010E969A8BEE
:10132000898BEDE7F2E0FC8BEB8BF3E0FD8BEB8937
:10133000FC8900808B899C8901969C8B8B8BE98929
:10134000FA89008289899A8901969A8B898B9D896D
:1013500091509D8BED89EE2351F780915E03909122
:101360005F032EE130E0B9010E940E17CB019B8391
:101370008A838A819B81992314F41B821A82CE016D
:1013800004962A813B814AE050E0BC01C9010E94D9
:10139000C916CE010496DC01FD0101900020E9F799
:1013A0003197CF018A1B9B0B8983109251031CC07C
:1013B00080915103082F112780915103282F332743
:1013C000CE010496FC01E20FF31F80810E948A087F
:1013D000282FCE010996FC01E00FF11F2083809198
:1013E00051038F5F8093510380915103282F33273E
:1013F0008981992787FD909528173907CCF2CE016E
:101400000E9623E0AC016EE082E00E94EC0529819B
:10141000998185E0382F391BCE010996AC016EE029
:10142000832F0E94EC0565960FB6F894DEBF0FBEC1
:10143000CDBFDF91CF911F910F910895CF93DF938F
:10144000CDB7DEB729970FB6F894DEBF0FBECDBF7C
:1014500080916603909167038E5590409C838B83A7
:101460008B819C8123E030E0B9010E940E17CB01F3
:101470009A83898389819A818A30910524F089E051
:1014800090E09A83898389819A81992314F41A823E
:10149000198220918C0230918D0289819A81821764
:1014A000930709F4D7C089819A81823091052CF481
:1014B00060E184E00E94B50104C060E084E00E9425
:1014C000B50189819A8190938D0280938C0280E886
:1014D0008D8384E88E8388E88F8389819A819987B8
:1014E0008887888599858430910509F45FC088854F
:1014F000998585309105DCF4888599858130910541
:1015000009F43FC088859985823091052CF488853F
:101510009985009779F173C0888599858230910506
:10152000B9F18885998583309105C9F168C08885AE
:1015300099858730910509F44EC088859985883052
:1015400091055CF48885998585309105B1F1888590
:10155000998586309105C1F152C08885998588307A
:10156000910509F43FC0888599858930910509F472
:1015700040C045C080E88D8384E88E8388E88F83EF
:101580003EC081E88D8384E88E8388E88F8337C0EE
:1015900082E88D8384E88E8388E88F8330C083E877
:1015A0008D8384E88E8388E88F8329C083E88D83C8
:1015B00085E88E8388E88F8322C083E88D8386E860
:1015C0008E8388E88F831BC083E88D8387E88E83B2
:1015D00088E88F8314C083E88D8387E88E8389E849
:1015E0008F830DC083E88D8387E88E838AE88F839D
:1015F00006C083E88D8387E88E838BE88F8360E065
:1016000085E00E94B50160E286E00E94B5018D810F
:10161000682F87E00E94B50160E085E00E94B50177
:101620006EE386E00E94B5018E81682F87E00E94FC
:10163000B50160E085E00E94B5016CE586E00E949E
:10164000B5018F81682F87E00E94B50160E084E0DA
:101650000E94B50129960FB6F894DEBF0FBECDBF2C
:10166000DF91CF910895CF93DF93CDB7DEB7269763
:101670000FB6F894DEBF0FBECDBF80915603909198
:10168000570326E130E0B9010E940E17CB01069600
:101690009E838D838D819E8199230CF446C08D811C
:1016A0009E812AE030E0B9010E940E17CB018A83A7
:1016B0008D819E812AE030E0B9010E940E17898356
:1016C000898186958C5F89838A81282F332786E8D4
:1016D00090E0821B930B9C838B8320910D013091B2
:1016E0000E018B819C818217930761F080910D011F
:1016F00090910E010E94EC0B8B819C8169810E946C
:10170000260C0AC0909199028981981729F08B8143
:101710009C8169810E94260C8981809399028B812A
:101720009C8190930E0180930D018D819E81992360
:101730000CF049C08D819E81909581959F4F9E832D
:101740008D838D819E812AE030E0B9010E940E17C1
:10175000CB018A838D819E812AE030E0B9010E940D
:101760000E1789838981869589838A8199278A576B
:101770009F4F9C838B8320910D0130910E018B81B3
:101780009C818217930761F080910D0190910E0169
:101790000E94EC0B8B819C8169810E94260C0AC0FF
:1017A000909199028981981729F08B819C81698198
:1017B0000E94260C8981809399028B819C81909351
:1017C0000E0180930D0126960FB6F894DEBF0FBE72
:1017D000CDBFDF91CF910895CF93DF93CDB7DEB723
:1017E00026970FB6F894DEBF0FBECDBF9E838D83C4
:1017F0001C821B821DC08D818A838D819E81892FD1
:1018000099278983698185E00E94B5016A8186E014
:101810000E94B50160E087E00E94B5018D819E8144
:101820004E969E838D838B819C8101969C838B83B6
:101830008B819C8188309105F0F226960FB6F89442
:10184000DEBF0FBECDBFDF91CF910895CF93DF9361
:10185000CDB7DEB727970FB6F894DEBF0FBECDBF6A
:101860009E838D836F831C821B8223C08D818A831C
:101870008D819E81892F99278983698185E00E94C6
:10188000B5016A8186E00E94B5018F819927FC012C
:10189000E35DFE4F8081682F87E00E94B5018D8156
:1018A0009E814E969E838D838B819C8101969C8325
:1018B0008B838B819C8188309105C0F227960FB66F
:1018C000F894DEBF0FBECDBFDF91CF910895CF93C7
:1018D000DF93CDB7DEB726970FB6F894DEBF0FBE05
:1018E000CDBF809154039091550326E130E0B901BA
:1018F0000E940E17CB019E838D838D819E8199233B
:101900000CF452C08D819E812AE030E0B9010E9422
:101910000E17CB018A838D819E812AE030E0B901C8
:101920000E940E1789838981869589838A81282F51
:10193000332787E090E0AC01421B530B9A018EE104
:1019400090E0AC01249FC001259F900D349F900D25
:1019500011240A969C838B8320910B0130910C01FA
:101960008B819C818217930761F080910B0190918C
:101970000C010E94370D8B819C8169810E949A0D18
:101980000AC0909198028981981729F08B819C81D7
:1019900069810E949A0D8981809398028B819C8134
:1019A00090930C0180930B018D819E8199230CF003
:1019B00055C08D819E81909581959F4F9E838D838B
:1019C0008D819E812AE030E0B9010E940E17CB0183
:1019D0008A838D819E812AE030E0B9010E940E1732
:1019E0008983898186958C5F89838A81282F332713
:1019F0008EE190E0AC01249FC001259F900D349FA3
:101A0000900D112486509F4F9C838B8320910B0156
:101A100030910C018B819C818217930761F080913A
:101A20000B0190910C010E94370D8B819C81698183
:101A30000E949A0D0AC0909198028981981729F006
:101A40008B819C8169810E949A0D89818093980283
:101A50008B819C8190930C0180930B0126960FB68D
:101A6000F894DEBF0FBECDBFDF91CF910895CF9325
:101A7000DF93CDB7DEB726970FB6F894DEBF0FBE63
:101A8000CDBF9E838D838D819E819C838B8318C067
:101A90008B818A838B819C81892F99278983698196
:101AA00085E00E94B5016A8186E00E94B50160E090
:101AB00087E00E94B5018B819C8101969C838B837A
:101AC0008D819E819C01275F3F4F8B819C81821776
:101AD0009307F0F280919802282F3327C901880FCD
:101AE000991F820F931FFC01EF5EFE4F80818823B8
:101AF000C1F08D819E8182969C838B838B818A83AA
:101B00008B819C81892F99278983698185E00E9437
:101B1000B5016A8186E00E94B50160E087E00E941D
:101B2000B50126960FB6F894DEBF0FBECDBFDF918C
:101B3000CF910895CF93DF93CDB7DEB727970FB638
:101B4000F894DEBF0FBECDBF9E838D836F838D81E2
:101B50009E819C838B8324C08B8189838B819C8114
:101B6000892F99278A836A8185E00E94B50169815E
:101B700086E00E94B5018F81282F3327C901880F85
:101B8000991F820F931FFC01E15FFE4F8081682F38
:101B900087E00E94B5018B819C8101969C838B8399
:101BA0008D819E819C01275F3F4F8B819C81821795
:101BB000930790F28D819E8104969C838B838B8109
:101BC00089838B819C81892F99278A836A8185E00B
:101BD0000E94B501698186E00E94B5018F81282F9E
:101BE0003327C901880F991F820F931FFC01E05F03
:101BF000FE4F8081682F87E00E94B5018F81282FDA
:101C00003327C901880F991F820F931FFC01EF5ED4
:101C1000FE4F8081882321F18D819E8182969C8355
:101C20008B838B8189838B819C81892F99278A83E0
:101C30006A8185E00E94B501698186E00E94B50154
:101C40008F81282F3327C901880F991F820F931F77
:101C5000FC01EF5EFE4F8081682F87E00E94B50196
:101C600027960FB6F894DEBF0FBECDBFDF91CF91A0
:101C70000895CF93DF93CDB7DEB760E085E00E9493
:101C8000B50163E886E00E94B50160E987E00E9443
:101C9000B50160E085E00E94B50164E886E00E943D
:101CA000B50161E987E00E94B50160E085E00E942E
:101CB000B50165E886E00E94B50162E987E00E940F
:101CC000B50160E085E00E94B50166E886E00E940B
:101CD000B50163E987E00E94B50160E085E00E94FC
:101CE000B50167E886E00E94B50164E987E00E94DB
:101CF000B50160E085E00E94B50168E886E00E94D9
:101D0000B50165E987E00E94B50160E085E00E94C9
:101D1000B50169E886E00E94B50166E987E00E94A6
:101D2000B50160E085E00E94B5016AE886E00E94A6
:101D3000B50167E987E00E94B50160E085E00E9497
:101D4000B50161EA86E00E94B50168E987E00E947A
:101D5000B50160E085E00E94B50162EA86E00E947C
:101D6000B50169E987E00E94B50160E085E00E9465
:101D7000B50163EA86E00E94B5016AE987E00E9446
:101D8000B50160E085E00E94B50164EA86E00E944A
:101D9000B5016BE987E00E94B50160E085E00E9433
:101DA000B50165EA86E00E94B5016CE987E00E9412
:101DB000B50160E085E00E94B50166EA86E00E9418
:101DC000B5016DE987E00E94B50160E085E00E9401
:101DD000B50167EA86E00E94B5016EE987E00E94DE
:101DE000B50160E085E00E94B50168EA86E00E94E6
:101DF000B5016FE987E00E94B50160E085E00E94CF
:101E0000B5016FEB86E00E94B50160EA87E00E94B1
:101E1000B50160E085E00E94B50160EC86E00E94BB
:101E2000B50161EA87E00E94B50160E085E00E94AB
:101E3000B50161EC86E00E94B50162EA87E00E948C
:101E4000B50160E085E00E94B50162EC86E00E9489
:101E5000B50163EA87E00E94B50160E085E00E9479
:101E6000B50163EC86E00E94B50164EA87E00E9458
:101E7000B50160E085E00E94B50164EC86E00E9457
:101E8000B50165EA87E00E94B50160E085E00E9447
:101E9000B50165EC86E00E94B50166EA87E00E9424
:101EA000B50160E085E00E94B50166EC86E00E9425
:101EB000B50167EA87E00E94B50160E085E00E9415
:101EC000B5016DED86E00E94B50168EA87E00E94E9
:101ED000B50160E085E00E94B5016EED86E00E94EC
:101EE000B50169EA87E00E94B50160E085E00E94E3
:101EF000B5016FED86E00E94B5016AEA87E00E94B5
:101F0000B50160E085E00E94B50160EE86E00E94C8
:101F1000B5016BEA87E00E94B50160E085E00E94B0
:101F2000B50161EE86E00E94B5016CEA87E00E948F
:101F3000B50160E085E00E94B50162EE86E00E9496
:101F4000B5016DEA87E00E94B50160E085E00E947E
:101F5000B50163EE86E00E94B5016EEA87E00E945B
:101F6000B50160E085E00E94B50164EE86E00E9464
:101F7000B5016FEA87E00E94B50160E085E00E944C
:101F8000B5016BEF86E00E94B50160EB87E00E942F
:101F9000B50160E085E00E94B5016CEF86E00E942B
:101FA000B50161EB87E00E94B50160E085E00E9429
:101FB000B5016DEF86E00E94B50162EB87E00E94FB
:101FC000B50160E085E00E94B5016EEF86E00E94F9
:101FD000B50163EB87E00E94B50160E085E00E94F7
:101FE000B5016FEF86E00E94B50164EB87E00E94C7
:101FF000B50161E085E00E94B50160E086E00E94E5
:10200000B50165EB87E00E94B50161E085E00E94C3
:10201000B50161E086E00E94B50166EB87E00E94B1
:10202000B501DF91CF910895CF93DF93CDB7DEB7A0
:1020300064970FB6F894DEBF0FBECDBF83E090E08B
:102040009C8B8B8B1A82198283E990E09C838B8313
:102050008091B602843409F0D5C0CFC08B899C89A9
:10206000FC01EC54FD4F80819927CD979A8B898B89
:102070008B899C8901969C8B8B8B8B899C89FC011D
:10208000EC54FD4F80819927CD97988B8F878B8952
:102090009C8901969C8B8B8B8B899C89FC01EC54D1
:1020A000FD4F80819927CD979E878D878B899C894D
:1020B00001969C8B8B8B8B899C89FC01EC54FD4F8A
:1020C00080819927CD979C878B878B899C890196E6
:1020D0009C8B8B8B89899A899C01220F331F220F3D
:1020E000331F8F85988995958795959587959595B3
:1020F000879595958795822B932B9A8789878F85CE
:1021000098898F7090709C0122953295307F32278C
:10211000207F32278D859E85959587959595879506
:10212000822B932B98878F838D859E8583709070EB
:102130009C0100243695279507943695279507949A
:10214000322F202D8B859C85822B932B9E838D8314
:102150008B819C8101979C838B838B819C812FEF4A
:102160008F3F920709F44EC089819A819C0180912A
:10217000800290918102F901E80FF91F898580831F
:1021800089819A8101969A8389838B819C810197A9
:102190009C838B838B819C812FEF8F3F920791F1E2
:1021A00089819A819C018091800290918102F9013C
:1021B000E80FF91F8F81808389819A8101969A8324
:1021C00089838B819C8101979C838B838B819C81EC
:1021D0002FEF8F3F9207B1F089819A819C01809106
:1021E000800290918102F901E80FF91F8D818083AF
:1021F00089819A8101969A8389838B819C8100973A
:1022000009F02CCF10929C0264960FB6F894DEBFB2
:102210000FBECDBFDF91CF910895CF93DF93CDB7A0
:10222000DEB7E9E2F0E082E28083E0E4F0E01082F1
:10223000E0E2F0E082E28083ECE5F0E01082A2E3ED
:10224000B0E0E2E3F0E0808181608C93A8E3B0E04D
:10225000E8E3F0E0808184608C93EAE2F0E088E9D2
:102260008083E0E4F0E086E88083EBE2F0E082EC5B
:102270008083E1E2F0E088E98083ECE5F0E086E845
:102280008083E2E2F0E082EC8083DF91CF910895D9
:10229000CF93DF93CDB7DEB764970FB6F894DEBF68
:1022A0000FBECDBF83E28F83188683E689871A86A7
:1022B0001B8685E090E09E838D831C821B821A82A0
:1022C000198215C029813A81CE010796FC01E20FDF
:1022D000F31F8081282F33278B819C81820F931FCE
:1022E0009C838B8389819A8101969A838983298132
:1022F0003A818D819E812817390724F38B819C8137
:1023000020E030E1B9010E940E179C838B838D8100
:102310009E819A8B898B8B819C819C8B8B8B8B89EB
:102320009C8999232CF48B899C89CF969C8B8B8BD1
:102330008B899C89082E892F000C881F990B000C13
:10234000881F991F282F235CCE010796E989FA89F7
:10235000E80FF91F20838D819E8101969E838D83D6
:10236000ED81FE818B819C8120E430E0B9010E94E7
:102370000E17282F235CCE010796E80FF91F208344
:102380008D819E8101969E838D832D813E81CE011C
:102390000796FC01E20FF31F8DE080838D819E8103
:1023A00001969E838D831A8219820FC029813A81FA
:1023B000CE010796FC01E20FF31F80810E94F3110A
:1023C00089819A8101969A83898389819A8188304B
:1023D000910564F364960FB6F894DEBF0FBECDBFCF
:1023E000DF91CF910895CF93DF93CDB7DEB72197DB
:1023F0000FB6F894DEBF0FBECDBF8983E2E2F0E0F6
:1024000080819927807290700097C1F3E3E2F0E039
:102410008981808321960FB6F894DEBF0FBECDBFB1
:10242000DF91CF910895CF93DF93CDB7DEB721979A
:102430000FB6F894DEBF0FBECDBF8983EBE2F0E0AC
:1024400080819927807290700097C1F3ECE2F0E0F0
:102450008981808321960FB6F894DEBF0FBECDBF71
:10246000DF91CF910895CF93DF93CDB7DEB7269755
:102470000FB6F894DEBF0FBECDBF9E838D838D81D6
:102480009E81DC01FD0101900020E9F73197CF0129
:102490008A1B9B0B9C838B831A8219820FC0298114
:1024A0003A818D819E81F901E80FF91F80810E9498
:1024B000131289819A8101969A83898329813A81AD
:1024C0008B819C818217930750F7809182020E9432
:1024D0001312809183020E94131226960FB6F8946D
:1024E000DEBF0FBECDBFDF91CF910895CF93DF93B5
:1024F000CDB7DEB72C970FB6F894DEBF0FBECDBFB9
:102500009C878B878B859C854AE050E09E012F5FDE
:102510003F4FB9010E94C916CE0101960E943312A5
:102520002C960FB6F894DEBF0FBECDBFDF91CF91D2
:102530000895CF93DF93CDB7DEB722970FB6F89407
:10254000DEBF0FBECDBF8A8387E089831FC08A812B
:10255000482F55278981282F332727FD309581E083
:1025600090E0022E02C0880F991F0A94E2F784239C
:1025700095231816190624F481E30E94131203C050
:1025800080E30E9413128981815089838981882385
:10259000F4F6809182020E941312809183020E94BD
:1025A000131222960FB6F894DEBF0FBECDBFDF9197
:1025B000CF9108951F920F920FB60F9211242F936F
:1025C0003F938F939F93AF93BF93EF93FF93CF93DB
:1025D000DF93CDB7DEB72297DEBFCDBFE3E2F0E0F9
:1025E000808180939403809194038D30D1F4809105
:1025F0009B028130B1F4A5E3B0E0E5E3F0E0808137
:10260000877F8C9310929B0281E080939C02809143
:102610004C03992720919403FC01EC54FD4F208337
:1026200048C080919B02282F33273A8329838981D0
:102630009A81009731F029813A812130310521F1C9
:1026400038C080919403833271F480919C02882376
:1026500051F481E080939B02A5E3B0E0E5E3F0E074
:10266000808188608C9310924C0330914C03832FAF
:10267000992720919403FC01EC54FD4F2083832F74
:102680008F5F80934C0315C080914C039927209154
:102690009403FC01EC54FD4F208380914C03863958
:1026A00030F480914C038F5F80934C0302C01092F2
:1026B0009B022296F894DEBFCDBFDF91CF91FF91B0
:1026C000EF91BF91AF919F918F913F912F910F907B
:1026D0000FBE0F901F901895CF93DF93CDB7DEB745
:1026E0006E970FB6F894DEBF0FBECDBF2091540396
:1026F00030915503CE010B964AE050E0BC01C90170
:102700000E94C91680E4898384E48A8380E38B83F2
:102710001C82CE010B96DC01FD0101900020E9F73F
:102720003197CF018A1B9B0B9E01255F3F4FAC0168
:10273000B901CE0101960E94B916CE010196DC01C5
:10274000FD0101900020E9F731979F012A1B3B0B07
:10275000CE010196820F931FFC0183E290E09183EA
:102760008083CE0101960E9433122091560330914E
:102770005703CE010B964AE050E0BC01C9010E940C
:10278000C91680E4898384E48A8381E38B831C8275
:10279000CE010B96DC01FD0101900020E9F7319795
:1027A000CF018A1B9B0B9E01255F3F4FAC01B901F6
:1027B000CE0101960E94B916CE010196DC01FD0101
:1027C00001900020E9F731979F012A1B3B0BCE01B6
:1027D0000196820F931FFC0183E290E09183808336
:1027E000CE0101960E94331220915E0330915F0367
:1027F000CE010B964AE050E0BC01C9010E94C91607
:1028000080E4898388E68A838DE38B831C82CE01F2
:102810000B96DC01FD0101900020E9F73197CF0113
:102820008A1B9B0B9E01255F3F4FAC01B901CE0176
:1028300001960E94B916CE010196DC01FD010190BE
:102840000020E9F731979F012A1B3B0BCE0101962F
:10285000820F931FFC0183E290E091838083CE017D
:1028600001960E9433122091660330916703CE01D6
:102870000B964AE050E0BC01C9010E94C91680E4F1
:10288000898386E58A838CE68B831C82CE010B9636
:10289000DC01FD0101900020E9F73197CF018A1B8F
:1028A0009B0B9E01255F3F4FAC01B901CE01019604
:1028B0000E94B916CE010196DC01FD0101900020B5
:1028C000E9F731979F012A1B3B0BCE010196820F3E
:1028D000931FFC0183E290E091838083CE010196F7
:1028E0000E9433122091B2023091B302CE010B96B6
:1028F0004AE050E0BC01C9010E94C91680E4898306
:102900008BE48A8387E68B831C82CE010B96DC01E5
:10291000FD0101900020E9F73197CF018A1B9B0B45
:102920009E01255F3F4FAC01B901CE0101960E9487
:10293000B916CE010196DC01FD0101900020E9F7F6
:1029400031979F012A1B3B0BCE010196820F931FEB
:10295000FC0183E290E091838083CE0101960E9486
:1029600033126E960FB6F894DEBF0FBECDBFDF9167
:10297000CF910895CF93DF93CDB7DEB7A5E3B0E055
:10298000E5E3F0E0908182E089278C93DF91CF919D
:102990000895CF93DF93CDB7DEB780918B0281305E
:1029A00041F4A5E3B0E0E5E3F0E0908181E0892720
:1029B0008C93DF91CF9108951F920F920FB60F92D3
:1029C00011242F933F934F935F936F937F938F9334
:1029D0009F93AF93BF93EF93FF93CF93DF93CDB7C5
:1029E000DEB780919D0290919E020097B1F4E4E4DD
:1029F000F0E0808191819093A4028093A302AEE4E1
:102A0000B0E0EEE4F0E080818F7B8C9381E090E099
:102A100090939E0280939D026FC0E4E4F0E0808179
:102A200091819093A2028093A102AEE4B0E0EEE423
:102A3000F0E0808180648C932091A1023091A20209
:102A40008091A3029091A402A901481B590BCA01CD
:102A50009093A00280939F0210929E0210929D027A
:102A600080919F029091A002865698409093A00278
:102A700080939F0280919F029091A0022CE231E00E
:102A8000B9010E94FA16CB019093A00280939F0295
:102A900080919F029091A002992324F41092A002A9
:102AA00010929F0280919F029091A0028730910521
:102AB00034F086E090E09093A00280939F02809192
:102AC0000101282F332727FD309580919F02909197
:102AD000A0022817390781F080919F029091A002EF
:102AE000863091054CF480919F029091A0028093D2
:102AF000010181E080939202DF91CF91FF91EF91EC
:102B0000BF91AF919F918F917F916F915F914F9105
:102B10003F912F910F900FBE0F901F901895CF935C
:102B2000DF93CDB7DEB780915E0390915F03909302
:102B30004B0380934A0320914A0330914B038091C9
:102B4000AE029091AF02A901481B590BCA019093A4
:102B5000AD028093AC0280914A0390914B03909315
:102B6000AF028093AE022091AA023091AB02809115
:102B7000AC029091AD02820F931F9093AB028093B1
:102B8000AA02809194028F5F8093940280919402B4
:102B90008630B1F4109294028091AA029091AB0217
:102BA00025E030E0B9010E940E17CB019093B102ED
:102BB0008093B0021092AB021092AA020E94B10858
:102BC000DF91CF9108951F920F920FB60F921124AB
:102BD0008F939F93AF93BF93EF93FF93CF93DF9325
:102BE000CDB7DEB7E3E4F0E010828091B0029091BF
:102BF000B102009741F0A2E3B0E0E2E3F0E090819F
:102C000088E089278C93DF91CF91FF91EF91BF915D
:102C1000AF919F918F910F900FBE0F901F901895BD
:102C20001F920F920FB60F9211242F933F934F9341
:102C30005F936F937F938F939F93AF93BF93EF9324
:102C4000FF93CF93DF93CDB7DEB78091A5028823A2
:102C5000D1F4E0E8F0E0808191819093A702809325
:102C6000A602AAE8B0E0EAE8F0E080818F7B8C93CE
:102C700081E08093A502A2E3B0E0E2E3F0E080818E
:102C800080618C9363C0E8E8F0E011821082E0E894
:102C9000F0E0808191819093A9028093A802AAE834
:102CA000B0E0EAE8F0E0808180648C931092A502A5
:102CB000A2E3B0E0E2E3F0E080818F7E8C9320918C
:102CC000A8023091A9028091A6029091A702A901C1
:102CD000481B590BCA019093A9028093A8028091C6
:102CE000A8029091A9028A5F90409093A9028093D4
:102CF000A8028091A8029091A90229E130E0B901CF
:102D00000E94FA16CB019093B3028093B202809195
:102D1000B2029091B30251E08836950730F087E611
:102D200091E09093B3028093B2028091A8029091B7
:102D3000A9022AEF30E0B9010E94FA16CB01909364
:102D40004E0380934D0381E080939502DF91CF91F4
:102D5000FF91EF91BF91AF919F918F917F916F9173
:102D60005F914F913F912F910F900FBE0F901F9049
:102D70001895FB01DC010D900020E9F711974150F7
:102D8000504028F0019000200D92C9F708951C9240
:102D90000895FB019F01E8944230C4F04532B4F439
:102DA0004A3029F497FB1EF4909581959F4F642F2C
:102DB00077270E94FA16805D8A330CF0895D819333
:102DC000CB010097A1F716F45DE251931082C9017F
:102DD0000C94EA16DC01FC0101900020E9F732971F
:102DE000AE17BF0730F47C916081708331976D938B
:102DF000F7CF0895AA1BBB1B51E107C0AA1FBB1F39
:102E0000A617B70710F0A61BB70B881F991F5A9576
:102E1000A9F780959095BC01CD01089597FB092EE7
:102E200007260AD077FD04D0E5DF06D000201AF48B
:102E3000709561957F4F0895F6F7909581959F4F16
:022E40000895F3
:102E4200010200000A310000440000230023005464
:102E520064665363655262005161005060005060C5
:102E62000051610052620053636554646667686989
:102E72006A6B6B6A69686755555555555555555571
:102E820055555555555555555555555555555555F0
:102E9200555555555555555555555555555500008A
:102EA20000AAAAAA00000055555555555555555525
:102EB2005555555555555555005554AA1552AA857F
:102EC200529685529685529685529685529685528D
:102ED200968552AA8554AA15550055555555000098
:102EE20000AAAAAA0AAAA052AA8554AA15555555FB
:102EF2005555555555555555005554AA1552AA853F
:102F020052958552955552AA1554AA855502855255
:102F1200568552AA8550AA055500155555550000EB
:102F220000AAAAAA0AAAA052AA8554AA15555555BA
:102F3200555555555555555055054A14A14A14A194
:102F42004A14A14A14A14A28A1522885522885521E
:102F5200828552828552828554001555555500004E
:102F620000AAAAAA0AAAA052AA8554AA155555557A
:102F7200555555555555555055054A14A14A84A1E4
:102F82004A80A14AA0A14A28A14A28A14A0AA14AE4
:102F920002A14A12A14A14A15055055555550000E7
:102FA20000AAAAAA0AAAA052AA8554AA155555553A
:102FB20055555555555555000000000000000000BC
:042FC20052030D0A9F
:00000001FF
